:020000020000FC
:1000000000C001E302BB00E007BB00E001BB02E06F
:100010000EBF0FE50DBF07E109B9539A549AE8D70F
:10002000809902C0A3D6AAD7E2D72FD26FEFB5D15D
:100030004CD0FBCFE395C8953196002009F0089588
:1000400050E0BFC1F9E0EAE3F6DF091679F4F3DF27
:10005000081669F4F0DF071659F43196C895002D9B
:100060003196C895F02DE02F099508953196319677
:100070003396EACF90EF80EF21E0088166D15130CE
:1000800011F41AD0F7CF702F17D00D3091F0952EB4
:1000900008815BD10D3069F0951639F4982F872FC0
:1000A000702F0AD02395233099F708814ED19516E9
:1000B00009F0089501D0F9CFD81529F4C71519F41E
:1000C00054E07FC1089521970895D0E0C8EC0AE874
:1000D000702E00E0802E088138D1523009F476C0AD
:1000E000D4D1A16001C0AE7F3DB7383010F458E0E4
:1000F00068C1C0DF7D30B9F0092D023031F49F7046
:100100008F707F7024D220D0EFCF9F758F757F7551
:10011000213029F4092D033011F407D0E5CF92DF07
:100120007D3009F00895A160089571547A3112F07C
:1001300055E047C17059A0FF11F406D00895F0E0D2
:10014000E72F708101D00895F1E0E62F70836A9562
:10015000633F10F456E035C108956395603012F0A6
:1001600057E02FC1F1E0E62F708108955BE029C1CF
:10017000D0E0C8ECFF24EE247727BF7D0881CA9524
:10018000E3940D3041F0E1D0523039F0B06251309B
:10019000A9F3F394F3CF0F2D0895B5FF7395EECF28
:1001A00054E00FC152E00DC19F708F707F70CFD1AE
:1001B0000895D0E0C8ECE93CA9F3088100833197A9
:1001C00021970D30C1F75E2E6F2E0895D1DF743068
:1001D00068F6062D013021F4052D033F09F452C0C5
:1001E000D0E0C8EC772788279927C715CAF208817D
:1001F000ACD0523029F4982F872F702F2197F5CF4C
:10020000D3DFA72EF62DE52DB77FBF7E9927882750
:100210007727BB243196F13011F4E43F59F0008187
:1002200094D0543039F0523089F7B394782F892F15
:10023000902FF0CF0B2D033029F0B394782F892F16
:1002400090E0F8CFB4FD02C0B061E0CFADDFA716FB
:1002500091F118F4B860DF2ECE2EF13021F4E43F96
:1002600011F4B3FF0FC0B3FF08C07A1508F442C001
:10027000F13019F4E43F09F43DC0F13039F6E43FC0
:1002800029F6089575DF003009F40895D0E0C8EC30
:10029000F62DE52DF03019F4E93C09F409C0088188
:1002A0000083319721970D30A9F75E2E6F2E0895A8
:1002B00002E0502F86C03197DF2FCE2FD03019F4B7
:1002C000C93C09F46DCF088121970D30B9F70E2F85
:1002D0000C1B500E08F46394D03011F4C93C29F083
:1002E0000881008321973197F7CF42DF003009F072
:1002F0006DCF08953DDF003039F1062D003021F437
:10030000052D095C0E15A0F2F62DE52DDF2FCE2F61
:10031000CE19D0400C2F502E0D2F602EFD1519F444
:10032000EC1509F405C00081088321963196F6CFBB
:10033000D0E0C8ECFD2DEC2D3197088100830D3005
:1003400019F031972197F9CF08955527102F1D30B7
:1003500009F416C01F75103009F402C01C3011F4E6
:1003600051E0089510310AF408951B350AF00895FC
:10037000103412F053E008951A310AF452E008954F
:1003800054E00895C83C19F427E075D00AC0212F25
:1003900081D0C3951DE0188304C02EE36CD0D0E05B
:1003A000C8EC7DD0183071F318831D3049F0CB387C
:1003B00019F427E060D0F5CFCA95212F6BD0F1CF8B
:1003C000089563D0503021F4F6E0E4E66CD042C0EA
:1003D000513021F4F6E0ECE866D03CC0523021F414
:1003E000F6E0EAEC60D036C0533021F4F6E0ECEEF3
:1003F0005AD030C0543021F4F7E0EEE254D02AC095
:10040000553021F4F7E0E0E64ED024C0563021F418
:10041000F7E0E4E948D01EC0573021F4F7E0E6EDFC
:1004200042D018C0583021F4F8E0E6E33CD012C0C6
:10043000593021F4F8E0E6E936D00CC05A3021F406
:10044000F8E0EEEC30D006C05B3021F4F9E0E6E0F5
:100450002AD000C00FE502E00EBF0FE50DBF6FEF21
:10046000A0E0B0E012D0E1CD57D0242F04D0232F4C
:1004700002D00895202F5D9BFECF55D6B6FF03C056
:100480005F9BFECFBF7B2CB908952DE0F4DF2AE0FF
:10049000F2DF08952D3011F4F8DF0895ECCF5F9B63
:1004A000FECF1CB10895C895002021F0202DE3DF78
:1004B0003196F9CF0895F7DFE8DF08954EDE07E0C3
:1004C00007174AF001E0703019F0000F7A95FBCF62
:1004D000702F3ADE08955AE074DF903039F0905D65
:1004E000292FC9DF803011F420E3C5DF803019F0F7
:1004F000805D282FC0DF705D272FBDDF089599270D
:100500008827745610F09395FCCF7C597A5010F0E0
:100510008395FCCF765F0895432F46954695469583
:100520004695405D4A3308F0495F3F70305D3A338D
:1005300008F0395F089546FD475F4F7036FD375F1D
:100540003F70440F440F440F440F342B08959330F1
:10055000B2F4923032F0863092F4853012F0763078
:1005600072F4882321F00AE0700F8A9581F79923AD
:1005700009F4089504E68894700F9A95C0F751E045
:1005800020CF83DF82DFF5E0EEE895DF08952020BD
:10059000202020204154544F424153494320766546
:1005A0007273696F6E20383531352D30323131310B
:1005B00035432E204E6F7420666F7220636F6D6D11
:1005C00065726369616C207573652E200A0D2020A9
:1005D00020202020436F7079726967687420323060
:1005E000303220627920526963686172642043610D
:1005F0007070656C7320616C6C20726967687473CD
:100600002072657365727665642E0A0D20202020A5
:100610002020687474703A2F2F70726F6A6563744B
:10062000732E63617070656C732E6F72672020206B
:100630002020202070726F6A65637473406361705C
:1006400070656C732E6F72670A0D000046726565E7
:10065000202070616765733A000020206368617232
:10066000733A00004572726F7220303A20556E6BFB
:100670006E6F776E20636F6D6D616E64206F722098
:100680006F70657261746F722E2000004572726F18
:100690007220313A20456E636F756E7465726564C1
:1006A00020612076616C75652074686174206973BF
:1006B000206E6F74206265747765656E20302061EE
:1006C0006E64203235352E2000004572726F722024
:1006D000323A2050726F6772616D206D656D6F7276
:1006E000792069732066756C6C2E00004572726FFC
:1006F0007220333A20456E636F756E74657265645F
:10070000206120636861726163746572207468613E
:1007100074206973206E6F742061207265636F6747
:100720006E697A656420747970652E2000004572C8
:10073000726F7220343A28696E7465726E616C2033
:100740006572726F72202D627566666572206C69C3
:100750006D697420657863656564656429200000AF
:100760004572726F7220353A20496E617070726FF7
:10077000707269617465207661726961626C65206E
:100780006E616D6520656E636F756E74657265640C
:100790002E2000004572726F7220363A2044617438
:1007A0006120737461636B20707573682065727269
:1007B0006F72202D746F6F206D616E79206172678A
:1007C000756D656E7473206F6E206F6E65206C6939
:1007D0006E652E2000004572726F7220373A2044F9
:1007E00061746120737461636B20706F7020657237
:1007F000726F722E0A0D20202020202020202046FB
:10080000756E6374696F6E20747269656420746FAD
:100810002075736520612076616C75652074686150
:100820007420776173206E6F7420617661696C61EA
:10083000626C652E00004572726F7220383A204D4E
:10084000616368696E6520737461636B20657272A1
:100850006F720A0D20202020202020202046756E57
:100860006374696F6E7320616E642F6F72206361B1
:100870006C6C73206E657374656420746F6F206494
:100880006565706C79206F7220746F6F20636F6D77
:10089000706C657800004572726F7220393A20479B
:1008A0004F544F206F7220474F5355422064657359
:1008B00074696E6174696F6E206C696E6520776112
:1008C00073206E6F7420666F756E642E0000457223
:1008D000726F7220413A205370656369666965647E
:1008E0002062697420706F736974696F6E20726121
:1008F0006E6765206F6620302E2E37206578636521
:100900006564656400004572726F7220423A204C43
:10091000696E65206E756D62657220686173206D09
:100920006F7265207468616E207468726565206EF0
:10093000756D6572616C732000004C49532082050F
:1009400053495A208E054E455720F70750500B202B
:10095000F50550500D20FC055052494EA20550524D
:100960005820A90550524220DB0650574D382B061F
:1009700050574520350650574F204106454D4954A4
:10098000CE06501A1D20B10550501D20BA05464F05
:10099000522058064E455854CB05501C1E20D405F5
:1009A00050501E20440650501C2025065049462019
:1009B0004E0650544F205A06505004205E065255A1
:1009C0004E20BE07454E44205C06414E442003069F
:1009D0004C5352200A064C534C200F06504F5220C5
:1009E0001406584F52201B0644554D500A08474FD5
:1009F000544F9006474F5355940652455455970609
:100A00005448454E54064B455920D30641434F2088
:100A1000E005534156459D064C4F4144B6065045AE
:100A2000454BE605504F4B45ED054F4441209B0794
:100A30004F4442209F074F444320A3074F44442084
:100A4000A7074F5041208B074F5042208F074F5030
:100A5000432093074F5044209707494E4120AB074E
:100A6000494E4220AE07494E4320B207494E44202A
:100A7000B50753424120E70643424120EE06534268
:100A80004220F60643424220FD065342432005071A
:100A9000434243200C07534244201407434244205E
:100AA0001B07534441202307434441202A07534452
:100AB0004220320743444220390753444320410730
:100AC00043444320480753444420500743444420B0
:100AD0005707494241205F07494242206A0749427D
:100AE0004320750749424420800744454C4127086C
:100AF0004453524548084453434F420844534445E5
:100B00003C080000C2DCF1E0E3EFF61511F4E51556
:100B100021F02081BFDC3197F8CFB7DCB6DCF6E0FE
:100B2000ECE4C1DC752D962D795C90400DDB792FBE
:100B3000E6DCD3DCF6E0EAE5B6DC0FDBE0DCCDDCBE
:100B4000A4DC0895AE7FD0DA08DBD9DCC6DC9DDCFE
:100B50000895C9DA24E28FDC00DB372F85DC95DCD1
:100B60000895AE7FC1DAF9DA072FF7DAF0E0E72F60
:100B700000830895A2FF40C0AE7FB6DAEEDAA72E5A
:100B8000ECDA872FEADAB72EF0E0E72F8083A06255
:100B9000A860AA7F0895F0E0EB2D00810A1519F0F6
:100BA00003950083A06108959EDAD7DA072FD5DA7E
:100BB000701719F07727C8DA08957FEFC5DA08951E
:100BC00092DA70E0459B71E0BFDA08958CDAC5DAFD
:100BD000E72FF0E07081B8DA089585DABEDA072FE2
:100BE000BCDAF0E0E02F708308957DDAB6DA072FE3
:100BF000B4DA700FA9DA089576DAAFDA072FADDA32
:100C0000701BA2DA08956FDAA8DA072FA6DA70232C
:100C10009BDA089568DAA1DA769596DA089563DAB0
:100C20009CDA770F91DA08955EDA97DA072F95DA72
:100C3000702B8ADA089557DA90DA072F8EDA702748
:100C400083DA089571E080DA08954DDA86DA072FA5
:100C500084DA70171EC047DA01E80FBD0EBD8D9A09
:100C60007CDA00E00BBD7ABD08953DDA03E80FBDE4
:100C700001E00EBDBD9A71DA072F6FDA7BBD0ABDA8
:100C8000089500E00FBD08952EDA67DA072F65DAC0
:100C9000071770E0BAF6B1F257DA089524DA5DDA90
:100CA000772309F0A26008950DB70E5F0DBF089578
:100CB000A460089518DA0895B26008954881FCD9B7
:100CC000388139DC732F40DAF7D90DDA08950BDA61
:100CD00044DA472FF1E0E3EF0AC0F61511F45E168F
:100CE000E8F400810D3011F03197F7CF3197772775
:100CF00088279927F61511F45E1680F4008125DB0C
:100D0000523029F4982F872F702F3197F3CF9F708F
:100D10008F707F701CDC471701F7089559E051CBA5
:100D2000D6DFDF2FCE2F0895D2DFA06C0895B2FF5B
:100D300002C0B1600895B26008956FEF752D04DAB6
:100D4000762D02DAD1E0CFEFEFEFF1E00881E19903
:100D5000FECFFFBBEEBB0DBBE29AE19AD03011F49F
:100D6000C93C19F031972197F1CF0895D1E0CFEF29
:100D7000EFEFF1E0E199FECFFFBBEEBBE09A0DB3E0
:100D80000883D03011F4C93C19F031972197F2CF84
:100D90006DEFE3D9672EE1D9572E0895A4D9DDD997
:100DA000272F69DB08955F9BFECF7CB1733009F478
:100DB000B260CAD9089597D9D0D908E020E3771F47
:100DC00008F421E358DB0A95C9F75FDB08958BD956
:100DD00075DBC3D90BB3072B02BB089584D96EDB37
:100DE000BCD970950BB3072302BB08957CD966DB91
:100DF000B4D908B3072B02BB089575D95FDBADD911
:100E0000709508B3072302BB08956DD957DBA5D9A8
:100E100005B3072B02BB089566D950DB9ED97095A8
:100E200005B3072302BB08955ED948DB96D902B308
:100E3000072B02BB089557D941DB8FD9709502B3B8
:100E4000072302BB08954FD939DB87D90AB3072B93
:100E50000ABB089548D932DB80D970950AB30723BD
:100E60000ABB089540D92ADB78D907B3072B07BB03
:100E7000089539D923DB71D9709507B3072307BBD0
:100E8000089531D91BDB69D904B3072B04BB08953E
:100E90002AD914DB62D9709504B3072304BB0895E3
:100EA00022D90CDB5AD901B3072B01BB08951BD9FA
:100EB00005DB53D9709501B307230ABB089513D9F5
:100EC000FDDA4BD909B3072370E0002309F471E080
:100ED0003BD9089508D9F2DA40D906B3072370E068
:100EE000002309F471E030D90895FDD8E7DA35D947
:100EF00003B3072370E0002309F471E025D90895B6
:100F0000F2D8DCDA2AD900B3072370E0002309F411
:100F100071E01AD90895E7D820D97BBB0895E3D8AA
:100F20001CD978BB0895DFD818D975BB0895DBD8D4
:100F300014D972BB0895D7D810D97ABB0895D3D8E5
:100F40000CD977BB0895CFD808D974BB0895CBD8F6
:100F500004D971BB089579B3F7D8089576B37C7F2F
:100F6000F3D8089573B3F0D8089570B37C7FECD8AC
:100F70000895427265616B200A0D0000D1E0C3EF55
:100F80006FEFA160D0D0A5FF03C0CC2EDD2EAF7DCA
:100F9000A4FF03C0DD2DCC2DAF7EA6FF03C0EC2E39
:100FA000FD2EAF7BA7FF04C0DF2FCE2FB460AF773D
:100FB000B0FF03C0DF2DCE2DBA7FB1FF04C043D0F8
:100FC000D62DC52DBD7FD61511F45C1678F4088199
:100FD000BCD9A1FF04C0543011F02197D1CFAD7F0F
:100FE000523011F42197CCCF7FD8CACF0895C9DAF7
:100FF00001E0602E03EF502EF62DE52D6FEFA0E0FF
:10100000B0E000E0F03011F4E93C19F000833197D2
:10101000F9CF0895F1E0E3EFF03011F4E93C41F04D
:10102000308122DA20E227DA20E225DA3197F4CF84
:101030002CDA2BDA362D18DA20E21DDA352D14DA07
:1010400024DA23DA0895FFE0E2E72DDA08954BD899
:1010500084D89927882755270027772361F09A9508
:101060008A955A954A95F1F70A95E1F7D1F7C1F7B4
:10107000B1F77A95F2CF089536D86FD8172F8894A4
:101080000BD0089530D869D8172F089405D008954B
:1010900027D0712F59D8089501B3077E01BB02B341
:1010A000086102BB99E0839BFECF949A8C9810F064
:1010B00094988C9A93988B9A2FD08B98939A2CD043
:1010C0008399F8CF18F0949A8C9802C094988C9ACF
:1010D000839BFECF8C98949A111F9A9521F70895BF
:1010E00001B3077D01BB02B3086102BB99E083999C
:1010F000FECF8894849B06C0089493988B9A849919
:10110000FECF04C093988B9A849BFECF8B98939AC2
:10111000111F9A9561F7089530E540E54A95F1F77A
:101120003A95D9F708955F9B09C00CB1033111F4CA
:0E113000B06404C00CB1033009F4B26008953D
:00000001FF
